:020000040800F2
:10000000B815002029020008E33200085D2F00081F
:10001000E132000869050008E5370008000000002B
:10002000000000000000000000000000E7320008AF
:100030001B06000800000000E5320008E932000855
:10004000430200084302000843020008430200087C
:10005000430200084302000843020008430200086C
:10006000430200084302000843020008430200085C
:1000700043020008430200089D05000843020008EF
:1000800043020008A90500084302000843020008D3
:10009000430200084302000843020008430200082C
:1000A000430200084302000843020008430200081C
:1000B0004302000843020008853300084302000899
:1000C00043020008430200084302000843020008FC
:1000D00043020008C1370008CD370008D9370008AF
:1000E00043020008430200084302000843020008DC
:1000F00043020008430200084302000843020008CC
:1001000000000000000000000000000043020008A2
:1001100043020008430200084302000843020008AB
:10012000430200084302000843020008430200089B
:100130004302000843020008000000000000000025
:1001400043020008430200084302000800000000C8
:10015000000000000000000000000000000000009F
:1001600000000000000000004302000843020008F5
:100170004302000800000000000000000000000032
:10018000000000004302000800F002F800F03CF814
:100190000AA090E8000C82448344AAF10107DA45E2
:1001A00001D100F031F8AFF2090EBAE80F0013F0F8
:1001B000010F18BFFB1A43F0010318473044000039
:1001C00050440000103A24BF78C878C1FAD85207CA
:1001D00024BF30C830C144BF04680C6070470000C1
:1001E0000023002400250026103A28BF78C1FBD840
:1001F000520728BF30C148BF0B6070471FB503F0DE
:10020000F6FA1FBD10B510BD00F0E2F81146FFF779
:10021000F5FF03F08FFD00F000F903B4FFF7F2FFE4
:1002200003BC00F007F9000009488047094800476F
:10023000FEE7FEE7FEE7FEE7FEE7FEE7FEE7FEE796
:10024000FEE7FEE704480549054A064B70470000F3
:100250007533000889010008B8050020B815002092
:10026000B80D0020B80D002053EA020C00F06980A0
:100270002DE9F04B4FF00006002B1FBFB3FA83F5BA
:1002800003FA05F424FA05F65E4012BF1643B2FAEB
:1002900082F502FA05F4C5F120051EBF22FA05FC1D
:1002A00044EA0C04203556EA044C4FEA144418BFC3
:1002B000641C4FF000084FF00009904271EB030CF2
:1002C00039D3002919BFB1FA81F701FA07F6B0FA5C
:1002D00080F700FA07F6C7F120071EBF20FA07FCD7
:1002E00046EA0C062037B6FBF4FCA7EB0507103FE7
:1002F00007F01F0BCBF120060CFA0BFB2CFA06F6CD
:1003000044BFB3460026202FA4BF5E464FF0000B2B
:100310005BEA060C08BF4FF0010B19EB0B09ABFBB6
:10032000027C48EB0608C01B06FB02CC0BFB03CC8F
:1003300071EB0C01C1E70B46024641464846BDE859
:10034000F08B13B54FF000004FF00001AFF30080C9
:10035000BDE81C407047B2F120030AD5C2F120036A
:1003600020FA02F001FA03F321FA02F140EA030055
:10037000704721FA03F04FF0000170474FF0000280
:1003800000B5134694469646203922BFA0E80C508B
:10039000A0E80C50B1F12001BFF4F7AF090728BF66
:1003A000A0E80C5048BF0CC05DF804EB890028BFE2
:1003B00040F8042B08BF704748BF20F8022B11F00B
:1003C000804F18BF00F8012B704770477047704787
:1003D000754600F02BF8AE4605006946534620F0FE
:1003E0000700854618B020B5FFF72CFFBDE8204078
:1003F0004FF000064FF000074FF000084FF0000BE1
:1004000021F00701AC46ACE8C009ACE8C009ACE893
:10041000C009ACE8C0098D46704710B50446AFF37B
:1004200000802046BDE81040FFF7F7BE0048704747
:100430005805002001491820ABBEFEE72600020047
:1004400070470146406A026C12F0500F03D0806B77
:10045000026B08461047016C41F4007101640168A9
:10046000C96811F4406F0CD1417E51B9016C21F47F
:1004700080710164016CC90403D4016C41F0010175
:10048000016400F057BB406A016C41F04001016417
:10049000416C41F00401416400F04EBB406A00F041
:1004A0004ABB000070B504460068816801F0030192
:1004B000012926D10168C90723D0816801F00D0107
:1004C000012910D1816841F0020181602168032077
:1004D000086000F0F3FF05460FE000BF00F0EEFFFC
:1004E000401B022809D9206C40F010002064606C89
:1004F00040F001006064012070BD20688068C00782
:10050000ECD1002070BD000070B504460068816821
:1005100001F00301012902D10168C90720D18168D6
:10052000104A11420DD1816841F00101816000F053
:10053000C5FF05460FE000BF00F0C0FF401B0228CA
:1005400009D9206C40F010002064606C40F001007C
:100550006064012070BD20680068C043C007EBD113
:10056000002070BD3F000080FEE770B505464FF6E5
:10057000FF7000224AF201040DE0AB5C58400023FA
:10058000C6074FEA500000D060405B1CDBB2082B6E
:10059000F6D3521CD2B28A42EFD370BD014800F0AC
:1005A0002BBD000068040020014800F025BD0000BC
:1005B000F00400200B4B01681422994207D20A4B29
:1005C0001944B1FBF2F189000164084908E0054BC8
:1005D0005B421944B1FBF2F1890001640149083919
:1005E000C163704708040240F8FFFDBF00000240ED
:1005F00030B590F840500124AC40C56B6C60046885
:1006000063604368102B036803D099600068C26080
:1006100030BD9A600068C16030BD704772B6FEE7B9
:1006200006490020C8610648016941F004010161E2
:10063000016941F040010161704700003805002068
:1006400000200240064A0021D16106490A6942F0B1
:1006500002020A614861086940F040000861704781
:100660003805002000200240044B0022DA61044AD1
:10067000136943F0010313610180704738050020BE
:10068000002002400A490020CA68D306094A04D55E
:10069000D06940F00200D0611020CB685B0705D51F
:1006A000D36943F00103D36140F00400C860704790
:1006B000002002403805002070B5054600F0FEFE1F
:1006C0000646104C09E0681C07D025B100F0F6FE84
:1006D000801BA84201D9032070BDE068C007F2D199
:1006E000E068800601D52020E060E068C00602D402
:1006F000E068400703D5FFF7C5FF012070BD00206B
:1007000070BD0000002002402DE9F041044690F841
:100710003C00884601280AD0012584F83C50204638
:10072000FFF7C0FE06004FF0000703D033E00220C1
:10073000BDE8F08125642068816821F080418160F6
:10074000B8F1010F04D12068816841F080418160D7
:100750002068816841F00041816000F0AFFE0546ED
:100760000FE000BF00F0AAFE401B0A2809D9206C48
:1007700020F0020040F01000206484F83C7001205A
:10078000D6E7206880680028ECDB206C20F00200AF
:1007900040F00100206484F83C703046C8E7000057
:1007A000F0B594B00024009490F83C202546012A2E
:1007B00019D0012780F83C7003689A6852077CD4EE
:1007C0004A681F26052A11D2D3F830C002EB420234
:1007D000520096402CEA060C0E6896404CEA060C35
:1007E000C3F830C035E0022014B0F0BD0A2A0FD2A1
:1007F000D3F834C0521F02EB4202520096402CEA5A
:10080000060C0E6896404CEA060CC3F834C020E093
:100810000F2A0FD2D3F838C00A3A02EB4202520034
:1008200096402CEA060C0E6896404CEA060CC3F87B
:1008300038C00EE0D3F83CC00F3A02EB420252003F
:1008400096402CEA060C0E6896404CEA060CC3F85B
:100850003CC00268936813F00C0F4FF0070374D18B
:10086000D1F800E0BEF10A0F10D39669AEF10A0E7E
:100870000EEB4E0C03FA0CFE26EA0E06D1F808E049
:100880000EFA0CFE46EA0E0696610FE0D2F814C08E
:100890000EEB4E0603FA06FE2CEA0E0CD1F808E029
:1008A0000EFA06FE4CEA0E0CC2F814C002684E693D
:1008B000D2F80CC0CCF3C10C00E0FDE04FEA4C0CC8
:1008C00006FA0CF6D1F810E0DFF848C2BEF1010FCD
:1008D00042D0BEF1020F4DD0BEF1030F58D0BEF191
:1008E000040F63D0166E91F800C006F0F846B6EB20
:1008F0008C6F03D1166E26F0004616660268566E9F
:1009000091F800C006F0F846B6EB8C6F03D1566E36
:1009100026F0004656660268966E91F800C006F012
:10092000F846B6EB8C6F03D1966E26F000469666BD
:100930000268D66E91F800C006F0F846B6EB8C6FF0
:1009400003D1D66E26F00046D6660268966806F099
:100950000306012E3AD136E0D2F860E00EEA0C0E22
:1009600091F800C046EA8C664EEA060E4EF000464C
:100970001666EAE7D2F864E00EEA0C0E91F800C0C1
:1009800046EA8C664EEA060E4EF000465666DCE7F6
:10099000D2F868E00EEA0C0E91F800C046EA8C66C8
:1009A0004EEA060E4EF000469666CEE7D2F86CE0B0
:1009B0000EEA0C0E91F800C046EA8C664EEA060E6E
:1009C0004EF00046C0E71668F6077AD1CE68012ED1
:1009D00006D052F8B03F0E78B740BB43136021E019
:1009E00052F8B06F91F800C007FA0CF73E4316605A
:1009F0000A680A2A0BD30668B769093A02EB420271
:100A000093409F438B6893401F43B7610AE0076898
:100A10007E69521C02EB420293409E438B689340D6
:100A20001E437E6103684FF0A0473B4EBB4201D09E
:100A3000B34201D1394A00E0394A0968102904D08B
:100A4000112907D012290AD03BE0D2F808C04FEA9A
:100A50000C2C08E0D2F808C04FEACC1C03E0D2F816
:100A600008C04FEA4C2CBCF1000F2ADBBB420DD072
:100A7000B34201D100970CE02A4EDFF8ACC0B3427C
:100A800002D1CDF800C004E0634501D1009600E03A
:100A900000959E6806F00306012E02D11E68F60737
:100AA0000AD1009E8EB1B66806F00306012E0CD165
:100AB000009E3668F60708D0016C41F02001016401
:100AC000012480F83C5020468EE6102908D01129D8
:100AD0001AD01229F5D1916841F480019160F0E7B4
:100AE000BB42EED1916841F4000191600F49104A78
:100AF0000968B1FBF2F101EB8101490000E0491EF8
:100B000000910029FBD1DCE7BB42DAD1916841F0CA
:100B10008071E3E700F0FF83000100500003005004
:100B2000000700500004005000050050580000204D
:100B300040420F007047704770470000F0B54FF01B
:100B4000000695B0040037463546009605D0206C67
:100B5000C00648D4206C18B133E0012015B0F0BDB8
:100B60006564E564A56484F83C50204600F00CF907
:100B700020688068C00024D42046FFF793FC064616
:100B8000206CC0061DD4E6B9206C20F4885040F0DB
:100B9000020020642068816821F040518160206853
:100BA000816841F0805181606E486F490068B0FBF8
:100BB000F1F000EB8000400000E0401E00900028B3
:100BC000FBD120688168C90002D5806880000AD501
:100BD000206C20F0020040F010002064606C40F0B7
:100BE000010060640126206CC00676D4002E74D10A
:100BF00020688168490770D4216C21F4807141F02C
:100C0000020121644FF0A04E584B704501D098422C
:100C100001D1574A00E0574ADFF85CC15749704597
:100C200001D100930EE0984202D1CDF800E009E036
:100C3000884202D1CDF800C004E0604501D10091A6
:100C400000E00095836803F00303012B02D10068E4
:100C5000C00710D1009840B1806800F0030001285F
:100C600003D100980068C00705D19068636820F43C
:100C7000403018439060D4E902201043626B012A8F
:100C800002D04FF4805300E00023627E43EA4233F7
:100C9000184394F820303843012B0AD1F2B1226C6A
:100CA00022F0020242F020022264626C42F0010251
:100CB0006264A26A012A21D023688B4201D0634575
:100CC00018D14FF430774FF4E071BA4213D04FF49B
:100CD00080739A420AD139460DE039E0A28C284B44
:100CE00003EB4242024342F48030E2E78A4201D100
:100CF000194600E011460143E06A084321688A680A
:100D000012F00C0F0BD1CA6844F202039A43CA6076
:100D1000217E94F83020890341EA42010843226889
:100D2000D168184B19400143D1602069012820681F
:100D3000016B21F00F0102D1E269521E11430163E0
:100D40006564206C20F0020040F00100206406E0A1
:100D5000206C20F0020040F0100020640126304694
:100D6000FCE600005800002040420F000001005047
:100D70000003005000070050000500500004005020
:100D80000000FEFF07C0F0FF70B586B005461421D5
:100D90006846FFF7F3FA1C492868884231D11B499D
:100DA000486940F080504861486900F080500590E3
:100DB000486940F4003048614869002600F400307A
:100DC0000590702000900320CDE9010669464FF0A0
:100DD000904000F089FA0F4C0D48C4E900068020CD
:100DE000C4E9026040002061800060612020C4E905
:100DF0000606204600F054F908B1FFF70FFCAC637B
:100E0000656206B070BD0000000100500010024095
:100E100008040240F80100202DE9F05F0446006854
:100E20008B469246816849077ED494F83C1001298C
:100E30000ED001214FF0A048DFF81091444F84F804
:100E40003C10404501D0B84205D1D8F8080304E071
:100E50000220BDE8F09FD9F800004FF0000610F026
:100E60001F0F01D0012504E02046FFF74DFB0500D0
:100E700002D084F83C6066E0206C40F60161884353
:100E800040F48070206420684146884201D0B84216
:100E900002D1D1F8082301E0D9F8002012F01F0F89
:100EA00004D0884202D02B4A904207D1216C21F411
:100EB00080112164C06880010ED413E0226C42F4DA
:100EC00080122264B84201D1C86802E021480C3087
:100ED000006810F0007F05D0206C20F4005040F432
:100EE00080502064206CC00404D5606C20F00600A3
:100EF000606400E0666484F83C60A16B1648886218
:100F0000A16B1648C862A16B1548086321681C20B4
:100F100008602068416841F0100141602068C168A4
:100F200041F00101C16000E00CE0216853465A46DF
:100F30004031A06B00F0DBF82068816841F00401CB
:100F4000816000E00225284683E700000807005082
:100F50000001005000040050430400089D040008F4
:100F60008704000810B590F821100022022905D04E
:100F70000421816380F82020012010BD01680B68E6
:100F800023F00E030B6001680B6823F001030B6074
:100F900090F84030C46B012101FA03F3636080F8DC
:100FA000211080F82020002010BD10B590F82110ED
:100FB0000024022903D004218163012418E0016880
:100FC0000A6822F00E020A6001680A6822F0010233
:100FD0000A6090F84020C36B012101FA02F25A60C6
:100FE00080F82110002180F82010416B01B1884762
:100FF000204610BD806B7047F0B4C16B0D6801686E
:101000000C68066C042202FA06F32B420FD0630729
:101010000DD50B689B0603D40B6823F004030B600B
:1010200090F840108A40C16B4A60C16A1BE00223FD
:1010300003FA06F72F424FF0000C4FF0010216D0D2
:10104000A70714D50C68A40605D40C6824F00A047C
:101050000C6080F8212090F840108B40C16B4B60F1
:1010600080F820C0816A002918D0F0BC0847082306
:10107000B3402B4212D0230710D50B6823F00E0388
:101080000B6090F84010C36B02FA01F15960826363
:1010900080F8212080F820C0016BE4E7F0BC7047A5
:1010A00070B5040021D0022084F821002268116864
:1010B00043F6F0708143D4E901031843D4E90335C2
:1010C0002B43184363691843A3691843E369184322
:1010D000084310602046FFF76DFA0020A06301214D
:1010E00084F8211084F8200070BD012070BD70B517
:1010F000044690F82000002501280CD0012084F837
:10110000200094F821600020012E06D084F82000F1
:101110000225284670BD022070BD022684F8216099
:10112000A0632068066826F0010606602046FFF7E7
:101130005FFAE06A00282068016802D041F00E01E1
:1011400006E041F00A0101602068016821F0040115
:1011500001602068016841F001010160D9E70000E9
:1011600070B5044600F0AAF90546601C02D0044898
:101170000078044400F0A2F9401BA042FAD370BDED
:101180004C0000202DE9F047054626480F46012671
:10119000017E01290FD00121814601762868DFF800
:1011A00088804CF25034012808D0A2462046FFF730
:1011B00083FAA0B130E00220BDE8F0872046FFF7B7
:1011C0007BFA00BBFFF72CFA2046FFF775FAD8F838
:1011D0001010064621F00401C8F810101CE04FF072
:1011E000FF3038606C6811E02046FFF72BFA50465C
:1011F000FFF762FAD8F81010060021F00201C8F8D3
:10120000101001D03C6007E004F50064D5E901014D
:1012100000EBC120A042E7D8002189F81810304621
:10122000CAE7000038050020002002400348016999
:1012300041F0800101610020704700000020024061
:101240002DE9F05F07461C4888460024017E1546BC
:101250001E46012909D00121814601764CF2503AFF
:101260005046FFF729FA18B122E00220BDE8F09FAE
:10127000012F02D0022F00D00427D346DFF83CA074
:10128000220128463146FFF766F881B208EB440098
:10129000FFF7EAF95846FFF70FFADAF8102022F0C4
:1012A0000102CAF8102018B9641CE4B2BC42E7D3AA
:1012B000002289F81820D9E73805002000200240D4
:1012C000064900200A69120607D5054A4A60054A00
:1012D0004A600969090600D50120704700200240D4
:1012E00023016745AB89EFCD2DE9FC4FDFF894A1D1
:1012F000002301250AF1040B03244FF00F0C0BF11E
:10130000040EB8E005FA03F632406FD04F68012FA3
:1013100005D0022F03D0112F01D0122F17D1D0F8F2
:1013200008905F0004FA07F829EA08090097D1F845
:101330000C8008FA07F848EA0908C0F808804768EE
:10134000B7430E79C6F300169E403E434660C6681A
:101350004FEA430804FA08F7BE4301978F6807FA7B
:1013600008F73743C7604E68022E01D0122E13D102
:10137000DE0800EB86060096366A5F07FF0E0CFA61
:1013800007F926EA0906D1F8109009FA07F949EA9F
:101390000609009EC6F820900668019FBE430F799B
:1013A00007F0030707FA08F7374307604E68F600AF
:1013B00060D5354EB76947F00107B761B66923F0CC
:1013C000030706F001060096304E3E44B146B6686B
:1013D0009F074FEA17780CFA08F7BE43B0F1904F19
:1013E00005D02B4FB84204D1012712E042E000277C
:1013F0000FE0284FB84201D102270AE0264FB84239
:1014000001D1032705E0254FB84201D1042700E0B0
:10141000052707FA08F73743C9F80870DAF80060BB
:101420005746D1F8048096435FEAC83800D5164382
:101430003E60DBF800605F46D1F8048096435FEAC7
:10144000883800D516433E60DEF800607746D1F854
:10145000048096435FEAC82800D516433E60094FD2
:101460000C373E68D1F8048096435FEA882800D59F
:1014700016433E605B1C0A6832FA03F67FF442AF03
:10148000BDE8FC8F00040140001002400000014054
:101490000004004800080048000C00480010004804
:1014A000426921EA02030A4043EA0241816170472E
:1014B0000AB181617047816270470000014880680D
:1014C000704700004C00002070B5040011D0216866
:1014D0004CF6CC400860216845F255500860D4E9CC
:1014E000000141602168A0688860FFF7E7FF0546BA
:1014F00009E0012070BD00BFFFF7E0FF401B262878
:1015000001D9032070BD2068C0680028F4D120688C
:101510000269E1688A4201D0016102E04AF6AA212B
:101520000160002070BD00684AF6AA210160002019
:10153000704700000248816802781144816070475A
:101540004C000020074810B5016841F0100101600F
:10155000032000F06DF8002000F006F800F024F8F9
:10156000002010BD0020024070B50D4D04464FF420
:101570007A712878B1FBF0F00A490968B1FBF0F004
:1015800000F074FD48B9102C07D200222146501EED
:1015900000F02EF800206C6070BD012070BD0000CE
:1015A0004C00002058000020094808B5816941F02E
:1015B00001018161816901F001010091C16941F07E
:1015C0008051C161C06900F08050009008BD0000EA
:1015D00000100240002809DB00F01F0201219140A9
:1015E0004009800000F1E020C0F8001170470000C1
:1015F000F0B40E4B1B680C46C3F30223C3F107057E
:10160000042D00D90425191D072901D2002300E06B
:10161000DB1E012606FA05F1491E214099409E4035
:10162000761E16403143F0BC02F0E0BA0CED00E04B
:10163000064900F0070208684FF6FF03184040EA29
:101640000220034A10430860704700000CED00E0E0
:101650000000FA05BFF34F8F05480168054A01F401
:10166000E06111430160BFF34F8F00BFFDE7000051
:101670000CED00E00400FA052DE9F84F044600687F
:101680000026804DC0036ED5E869C00008D4E86923
:1016900040F08050E861E869012600F08050009039
:1016A00079480168C90512D40168804641F4807107
:1016B0000160FFF703FF074605E000BFFFF7FEFEEE
:1016C000C01B642835D8D8F80000C005F6D5286AB4
:1016D00010F4407053D0A18801F4407181424ED083
:1016E000286A4FF4803191FAA1F2B2FA82F297009F
:1016F000664A4FF00108174420F44070C7F8008490
:1017000091FAA1F1B1FA81F102EB81010023C1F854
:1017100000342862C00732D0FFF7D0FE074641F2FE
:10172000883A4FF0020907E0FFF7C8FEC11B514598
:1017300002D90320BDE8F88F99FAA9F0B0FA80F039
:1017400040F040024946B8EB521F01D12A680CE034
:1017500091FAA1F2B2FA82F242F04002B1EB521FCA
:1017600002D12A6A01E015E06A6A99FAA9F1B1FA90
:1017700081F101F01F0108FA01F00242D4D0286A79
:10178000616820F44070084328621EB1E86920F0C7
:101790008050E8612078C00705D0286BA16820F050
:1017A0000300084328632078800705D5286BE1688B
:1017B00020F44030084328632078400705D5286B83
:1017C000216920F44020084328632078800605D54D
:1017D000286BE16920F0100008432863206880032B
:1017E00005D56868A16B20F4800008436860207804
:1017F000400605D5286B216A20F0200008432863A5
:101800002078000705D5286B616920F44010084353
:1018100028632078C00605D5286BA16920F4400014
:10182000084328632088800505D56868E16A20F4AC
:101830000000084368602078000605D5E86A616A00
:1018400020F4F8700843E8622088C00505D5E86AEE
:10185000A16A20F478500843E8622088C00405D5C6
:10186000286B216B20F48070084328632088800453
:1018700005D5286B616B20F40070084328630020B5
:1018800058E7000000100240007000400000424293
:101890002DE9F0470F46050069D04A4E306800F048
:1018A0000700B84209D2306820F0070038433060A2
:1018B000306800F00700B84259D12878424C8007C0
:1018C00005D56068A96820F0F000084360602878BA
:1018D000C0073DD06968012001290DD0022923D01D
:1018E0005FF0020393FAA3F2B2FA82F242F020020E
:1018F000520904D0226803E04FF40033F2E7626A31
:1019000093FAA3F3B3FA83F303F01F039840024260
:101910002DD0606820F0030008436060FFF7CEFD23
:10192000804641F288390CE04FF00073DAE700BFDF
:10193000FFF7C4FDA0EB0801494502D90320BDE82B
:10194000F0876068696800F00C00B0EB810FEFD1A0
:10195000306800F00700B8420BD9306820F007006B
:1019600038433060306800F00700B84201D00120F1
:10197000E5E72878400705D56068E96820F4E0606D
:10198000084360602878000706D56068296920F45C
:10199000605040EAC100606000F04EF86168F022DB
:1019A00092FAA2F201F0F001B2FA82F2D140074AB3
:1019B000515CC8400649086006480068FFF7D4FD3E
:1019C0000020BCE70020024000100240DA45000879
:1019D0005800002050000020084809490068496864
:1019E0004FF4E06292FAA2F201F4E061B2FA82F2FC
:1019F000D140044A515CC8407047000058000020A4
:101A000000100240F8370008084809490068496892
:101A10004FF4605292FAA2F201F46051B2FA82F2EB
:101A2000D140044A515CC840704700005800002073
:101A300000100240F8370008164A10B551681648E1
:101A400001F00C03042B20D0082B1ED14FF470148E
:101A500094FAA4F401F47013B4FA84F4E3400F4C44
:101A6000D26AE45C0F2393FAA3F302F00F02B3FAF5
:101A700083F3DA40094B1033C9039A5C06D500237F
:101A80001946FEF7F1FBA0FB040110BD0448A4FBBE
:101A9000000110BD0010024000127A00BA45000893
:101AA00000093D002DE9F84F050071D02878FC4E63
:101AB000C0074FF0010425D070686704C0F38100AF
:101AC000012807D07068C0F3810002281BD170681C
:101AD000C00318D597FAA7F0B0FA80F040F02000C4
:101AE000400901D0306800E0706A97FAA7F1B1FAB6
:101AF00081F101F01F0104FA01F1084265D0686824
:101B00000028D2D061E06868B0F5803F0BD010B1FA
:101B1000B0F5A02F17D0306820F4803030603068E6
:101B200020F4802002E0306840F480303060F06AB9
:101B3000A96820F00F000843F062686820B3FFF73F
:101B4000BDFC80460AE0306840F480203060EAE75F
:101B5000FFF7B4FCA0EB0800642871D897FAA7F04F
:101B6000B0FA80F040F02000400901D0306800E079
:101B7000706A97FAA7F1B1FA81F101F01F0104FA36
:101B800001F10842E4D020E0FFF798FC804607E02E
:101B9000C2E000BFFFF792FCA0EB08006428DCD88D
:101BA00097FAA7F0B0FA80F040F02000400901D089
:101BB000306800E0706A97FAA7F1B1FA81F101F09C
:101BC0001F0104FA01F10842E4D12878DFF8D48239
:101BD00080074FF0000A4FF0020730D570684FF0D1
:101BE000F80B10F00C0F07D07068C0F381000228CA
:101BF00027D17068C00324D497FAA7F0B0FA80F018
:101C000040F02000400901D0306800E0706A97FA87
:101C1000A7F1B1FA81F101F01F0104FA01F10842C4
:101C200002D02869012877D130689BFAABF220F006
:101C3000F8016869B2FA82F29040014331605AE0DB
:101C400064E1286988B394FAA4F0B0FA80F048F807
:101C50002040FFF733FC814606E000BFFFF72EFC73
:101C6000A0EB090002289AD897FAA7F0B0FA80F002
:101C700040F02000400901D0306800E0706A97FA17
:101C8000A7F1B1FA81F101F01F0104FA01F1084254
:101C9000E4D030689BFAABF26969B2FA82F220F0C4
:101CA000F80091400843306025E0FFE794FAA4F083
:101CB000B0FA80F048F820A0FFF700FC814605E06C
:101CC000FFF7FCFBA0EB09000228CCD897FAA7F09D
:101CD000B0FA80F040F02000400901D0306800E008
:101CE000706A97FAA7F1B1FA81F101F01F0104FAC5
:101CF00001F10842E4D1287800076CD5A869A8B39F
:101D000094FAA4F0B0FA80F008EB8000C0F88044A8
:101D1000FFF7D4FB814607E0A4E100BFFFF7CEFB4D
:101D2000A0EB090002289ED897FAA7F0B0FA80F03D
:101D300040F06000B4EB501F01D130680BE097FA1F
:101D4000A7F0B0FA80F040F06000B7EB501F01D16F
:101D5000306A00E0706A97FAA7F1B1FA81F101F0F8
:101D60001F0104FA01F21042D8D034E0FFE794FAE0
:101D7000A4F1B1FA81F108EB8101C1F880A4FFF769
:101D80009DFB814606E000BFFFF798FBA0EB090032
:101D900002289AD897FAA7F0B0FA80F040F06000D5
:101DA000B4EB501F01D130680BE097FAA7F0B0FAFE
:101DB00080F040F06000B7EB501F01D1306A00E0C6
:101DC000706A97FAA7F1B1FA81F101F01F0104FAE4
:101DD00001F21042D8D12878400768D5F0694FF059
:101DE0000009C00009D4F06940F08050F061F0694A
:101DF0004FF0010900F0805000902B480168C905A0
:101E000012D4016841F480710160FFF757FB8346EB
:101E100006E000BFFFF752FBA0EB0B00642875D86B
:101E200021480068C005F5D5E86801280AD008B146
:101E3000052811D0306A20F001003062306A20F0AD
:101E4000040002E0306A40F001003062E86868B3E4
:101E5000FFF734FB83460DE0306A40F00400306247
:101E6000F0E700BFFFF72AFBA0EB0B0141F288303F
:101E700081424BD897FAA7F0B0FA80F040F04000CA
:101E8000B4EB501F01D1306813E097FAA7F0B0FA15
:101E900080F040F04000B7EB501F09D1306A08E0F5
:101EA0000010024000004242007000400CE040E0A0
:101EB000706A97FAA7F1B1FA81F101F01F0104FAF3
:101EC00001F21042CED02DE0FFF7F8FA834607E08A
:101ED000FFF7F4FAA0EB0B0141F28830814215D8EC
:101EE00097FAA7F0B0FA80F040F04000B4EB501F32
:101EF00001D130680CE097FAA7F0B0FA80F040F01A
:101F00004000B7EB501F02D1306A01E083E0706AF5
:101F100097FAA7F1B1FA81F101F01F0104FA01F279
:101F20001042D5D1B9F1000F03D0F06920F08050F4
:101F3000F061E86980B37168C1F38101022977D04B
:101F40004FF080714F000228504609D091FAA1F15C
:101F5000B1FA81F148F82100FFF7B0FA05465DE0DB
:101F6000894691FAA1F1B1FA81F1C24648F82100FF
:101F7000FFF7A4FA804605E0FFF7A0FAA0EB0800FF
:101F8000022848D897FAA7F0B0FA80F040F0200075
:101F9000400902D0306801E066E0706A97FAA7F164
:101FA000B1FA81F101F01F0104FA01F10842E3D115
:101FB000D5E908100843716821F474110843706072
:101FC00099FAA9F0B0FA80F04AF82040FFF776FAC3
:101FD000054604E0FFF772FA401B02281BD897FA67
:101FE000A7F0B0FA80F040F02000400901D030683E
:101FF00000E0706A97FAA7F1B1FA81F101F01F01D0
:1020000004FA01F10842E5D02EE000BFFFF756FACE
:10201000401B022802D90320BDE8F88F97FAA7F0E9
:10202000B0FA80F040F02000400902D0306801E0B2
:102030000BE0706A97FAA7F1B1FA81F101F01F0184
:1020400004FA01F10842E1D10EE00128E4D0706801
:102050002A6A00F48031914204D1696A00F4701058
:10206000884201D00120D7E70020D5E710B5401EF7
:10207000B0F1807F01D3012010BD4FF0E0246061FA
:102080000F21601701F0B2FD0020A0610720206140
:10209000002010BD7047704770470000F0B590F801
:1020A0003C20012A36D0012480F83C40022280F8EE
:1020B0003D20026853689568174E184FB24201D010
:1020C000BA4204D123F4700C4B6843EA0C0323F0AA
:1020D000700C0B6843EA0C0353600268B2420DD0E7
:1020E000B2F1804F0AD00E4B9A4207D00D4B9A4264
:1020F00004D0BA4202D00C4B9A4204D1896825F030
:1021000080031943916080F83D40002180F83C1025
:102110000846F0BD0220F0BD002C01400034014013
:1021200000040040000800400040014010B50400D9
:1021300003D094F83D0010B107E0012010BD00204D
:1021400084F83C00204600F023F8022084F83D008B
:10215000211D206801F01CF9012084F8480084F852
:102160003E0084F83F0084F8400084F8410084F881
:10217000420084F8430084F8440084F8450084F861
:10218000460084F8470084F83D00002010BD0000A0
:1021900008B500680B49884212D10B48C16941F06B
:1021A0000401C161C069002200F004000090012117
:1021B0001E20FFF71DFABDE808401E20FFF70ABAEF
:1021C00008BD0000000800400010024090F83D10DB
:1021D000012901D001207047022180F83D100168DB
:1021E000CA6842F00102CA600068104988420ED0F5
:1021F000B0F1804F0BD00E49884208D00D4988427B
:1022000005D00D49884202D00C49884207D1816827
:102210000B4A1140062906D0B1F5803F03D0016872
:1022200041F001010160002070470000002C0140D6
:10223000000400400008004000340140004001401C
:102240000700010070B5044690F83C00012817D043
:10225000012584F83C50022084F83D0022689068F3
:102260002E4B184020F47F4090600868502830D0F2
:102270000DDC20284DD005DC98B310283BD148E078
:10228000022070BD302844D0402834D139E0602885
:1022900028D0702806D0B0F5805F2CD0B0F5005F54
:1022A00029D10AE0CB68D1E90121206801F0C8F802
:1022B0002068816841F0770109E0CB68D1E901210C
:1022C000206801F0BDF82068816841F48041816098
:1022D00011E0CA684968206801F0C4F850212068FC
:1022E00007E016E0CA684968206801F0CCF8602170
:1022F000206801F0AFF884F83D50002084F83C00DD
:1023000070BDCA684968206801F0ACF840212068B7
:10231000EFE7226801461046EBE7000088FFFEFF6A
:10232000704770B50446006801694FF00005C94365
:10233000890715D4C168C943890711D4E91E016111
:1023400001202077206880698007204602D0FFF7AF
:10235000E7FF04E000F0A7F8204600F0A5F8257795
:1023600020680169C943490717D4C168C9434907AF
:1023700013D46FF004010161022020772068806986
:1023800010F4407F204602D0FFF7CAFF04E000F0BF
:102390008AF8204600F088F8257720680169C9434B
:1023A000090716D4C168C943090712D46FF00801A0
:1023B0000161042020772068C0698007204602D090
:1023C000FFF7AEFF04E000F06EF8204600F06CF876
:1023D000257720680169C943C90617D4C168C94374
:1023E000C90613D46FF0100101610820207720681E
:1023F000C06910F4407F204602D0FFF791FF04E04F
:1024000000F051F8204600F04FF825772068016968
:10241000C943C90708D1C168C943C90704D1891E86
:102420000161204600F042F820680169C9430906AD
:1024300009D4C168C943090605D46FF08001016160
:102440002046FFF728FE20680169C943C90509D461
:10245000C168C943090605D46FF480710161204643
:10246000FFF718FE20680169C943490609D4C1680D
:10247000C943490605D46FF040010161204600F0D0
:102480003FF920680169C94389060BD4C168C94373
:10249000890607D46FF0200101612046BDE8704035
:1024A000FFF7FABD70BD7047704700002DE9F0419D
:1024B00000688E49884240D18E4E8D4DF168287853
:1024C0000978884237D100242746B1782846FEF79C
:1024D0004CF880BB6B7801224FF4004005F15001AD
:1024E000052B77D008DC012B29D0022B27D0032B1A
:1024F00040D0042B06D171E0062B6CD00F2B6BD093
:10250000102B6AD089206870AA700120FEF728FE7F
:102510000122794D140321462846FEF7C9FF4FF6E4
:10252000FF733A467249754800F070FC002221465C
:102530002846FEF7BDFF0020B070BDE8F081AB7803
:102540001C02EB7823431C0903F00F0331F814102D
:10255000D840C0B20142AA700AD0FF20E87004211E
:102560006348FEF702F82871000A68710627CCE775
:102570000020F3E7A878EB786A7943EA002328790A
:1025800042EA00225000A870002011E01F1805EB5D
:10259000040C31F817708CF80370641CE4B205EB7E
:1025A000040C3F0A641C401C8CF80370E4B2C0B2F7
:1025B0009042EBD3A878C01CC1B24D48FDF7D5FFBF
:1025C0002919641CC870E1B22944000AC870AF78A8
:1025D0007F1D9AE723E038E042E060E0A878EF78DA
:1025E0006B7947EA0027287943EA00235800A8704E
:1025F000002011E03A1805EB040C31F812208CF899
:102600000320641CE4B205EB040C120A641C401C99
:102610008CF80320E4B2C0B29842EBD3CAE7AA78A0
:102620001302EA781A432B79DB074FEA121302F000
:102630000F0231F8134020FA02F001D0044300E009
:10264000844321F81340B7785FE7A8786B790202DA
:10265000E87810432A7942EA032221F81020F2E7B1
:10266000A878EA786B7942EA00222879EC7943EA83
:102670000023002004E01718401C21F81740C0B2C6
:102680009842F8D38F2068700220A8700321184860
:10269000FDF76BFFE870000A2871052735E7A87879
:1026A000EF786B7947EA0027287943EA0023002076
:1026B00010E02A19641C92F807C0E2B2AC1807EBCC
:1026C000000EE479521C4CEA042421F81E40401C00
:1026D000D4B2C0B29842ECD306210548FDF745FFBD
:1026E000A871000AE87108270FE700000008004001
:1026F000B60000200000002000080048A0030020D1
:10270000704710B50446C06F20281CD181B17AB142
:1027100094F87400012816D0012084F87400206613
:10272000204601F091F9002803D1216E012901D042
:10273000012010BD22681021116221680A6842F050
:1027400010020A6010BD022010BD000070B50546E1
:102750000068104A90421BD1072912D10E4C2078F4
:1027600001280ED1607803280BD1A078022808D167
:102770002046FDF7FAFE20B9B4F80300074940BA35
:10278000C8802846BDE870400A220349FFF7B9BF58
:1027900070BD0000004400405C00002000000020EC
:1027A000704770B504460068016821F490710160BB
:1027B0002068816821F001018160206E012804D128
:1027C0002068016821F010010160206881684FF0E5
:1027D000000549060FD5816821F040018160206F16
:1027E00048B14563206FFEF7BDFB20B1206FFEF7B7
:1027F00001FC20280ED0A4F85A5021680F2008624E
:102800002068816941F0080181612020E067256628
:10281000002070BD1020C4F88000032070BD7047F8
:1028200070B504460068016821F490710160206869
:10283000816821F001018160206E012804D12068A7
:10284000016821F010010160216888684FF00F02D3
:1028500045064FF000004FF0200320D58D6825F08D
:1028600040058D60216F49B10F484863206FFEF726
:102870009CFB90B1206F416B88470EE0A4F85A0092
:10288000606521680A6221688A6942F008028A61EB
:10289000E36720662046FFF7C2FF002070BDA4F862
:1028A0005A0060650A62F3E7A5360008044A016829
:1028B000914203D10A220349FFF723BF704700006A
:1028C000004400405C0000202DE9F041026804460D
:1028D000D0691168936840F60F0528424FF0000553
:1028E00005D1860678D58E0676D5616EF2E0824FE8
:1028F00003F001060F4037437ED0C70709D0CF054C
:1029000007D501271762D4F8802042F00102C4F8ED
:10291000802082070AD5DA0708D0276802223A62A7
:10292000D4F8802042F00402C4F8802042070AD57F
:10293000DA0708D0236804221A62D4F8802042F013
:102940000202C4F8802002070CD501F020023243B5
:1029500008D0236808221A62D4F8802042F00802C6
:10296000C4F8802002050BD54A0109D523684FF42D
:1029700000621A62D4F8802042F02002C4F880205D
:10298000D4F88020002A2FD0800605D5880603D5EC
:10299000616E09B120468847D4F8800021688968B3
:1029A000490602D410F0280F20D0204600F0A9FEDE
:1029B00020688168490614D5816821F04001816052
:1029C000206F70B14D494163206FFEF7EEFA002889
:1029D0000AD0206F416B01E00EE02046BDE8F041D7
:1029E00008472046FFF762FFBDE8F0812046FFF769
:1029F0005DFFC4F88050F7E7276E2026012F58D1DD
:102A0000C70656D5CF0654D51020106222689068AC
:102A100040062DD5216F086840680004000CE3D003
:102A2000B4F858308342DFD9A4F85A0088692028C6
:102A300017D0106820F4807010602068816821F041
:102A4000010181602068816821F040018160E667B2
:102A500025662068016821F010010160206FFEF7F3
:102A600081FAB4F85800B4F85A10401A81B21CE048
:102A7000B4F85800B4F85A10401A81B2B4F85A00A9
:102A80000028B1D00029AFD0106820F490701060F9
:102A90002068826822F001028260E667256665662A
:102AA0002068026822F0100202602046FFF74EFE06
:102AB0009AE7C70209D55B0207D54FF48010106270
:102AC0002046BDE8F041FFF76BBE030605D50B06B7
:102AD00003D5A16E002980D186E7400684D548063B
:102AE00082D51168204621F040011160A667A566D5
:102AF00000F032FA78E7000020010004CF3500082A
:102B000010B5040002D0A06F10B107E0012010BD85
:102B1000002084F87400204600F026F82420A067E6
:102B20002068016821F001010160204600F0A8FE44
:102B30000128ECD0606A10B1204600F0B6FC206895
:102B4000416821F4904141602068816821F02A01A8
:102B500081602068016841F0010101602046BDE804
:102B6000104000F006BD00002DE9F04786B0044695
:102B700014216846FDF702FCDFF894812668654859
:102B8000022303210722002580274FF0010C4FF07C
:102B9000904A4FF01009464545D1866946F4804673
:102BA0008661866906F480460596466946F40036D5
:102BB0004661406900F400300590CDE903124802F7
:102BC0008DE8091069465046FEF78EFB534E524879
:102BD000C6E90005C6E9025735617561B561304641
:102BE000F561FEF75DFA08B1FDF718FD266774621E
:102BF0004A4E494844361438C6E902573561756172
:102C0000B561F561C6E900093046FEF749FA08B139
:102C1000FDF704FDE6660022022125207462FEF71E
:102C2000E7FC25204AE0DFF8F88046454BD1C6692D
:102C300046F40036C661C66906F400360596466954
:102C400046F400364661406900F400300590CDE955
:102C500003120C208DE8290069465046FEF744FB1C
:102C60002E4E2D4888361430C6E90005C6E90257B5
:102C700035617561B5613046F561FEF711FA08B14D
:102C8000FDF7CCFC26677462244E2348CC362830EE
:102C9000C6E9025735617561B561F561C6E900099C
:102CA0003046FEF7FDF908B1FDF7B8FCE6660022F4
:102CB000012126207462FEF79BFC2620FEF78AFC89
:102CC00006B0BDE8F087174CA642F9D1C46944F4B8
:102CD0008024C461C46904F480240594446944F4E4
:102CE00000244461406900F400200590CDE90312FE
:102CF0004FF440608DE8091069460B48FEF7F4FA7E
:102D0000002211462720FEF773FC2720D6E700009B
:102D10000038014000100240580002402404002006
:102D200000440040004800400008004830B4C36F31
:102D3000202B18D1A1B19AB190F87430012B12D088
:102D4000012380F874300023036603685C68240262
:102D500003D51C6844F080641C6030BC00F074BE75
:102D6000012030BC70470220FBE710B4C36F202B5A
:102D700018D1A1B19AB190F87430012B12D001236F
:102D800080F874300023036603685C68240203D56E
:102D90001C6844F080641C6010BC00F097BE0120E9
:102DA00010BC70470220FBE710B50068104988424C
:102DB0001DD11048104B8178C2785A545022491CBA
:102DC000B1FBF2F302FB131181700C490020086083
:102DD0000B48FFF725FD07490122C91C0848FFF7EA
:102DE000C4FF08480068016841F00101016010BD9E
:102DF0000048004000000020B600002024080040E9
:102E0000A00300204C020020704700002DE9F84389
:102E10000446806F1F4616460D4620284FD1CDB17F
:102E2000C6B194F87400012849D0012084F87400D8
:102E30004FF00008C4F880802120A067FEF73EFB19
:102E4000A4F850608146A4F85260A068B0F5805F95
:102E500003D004E00120BDE8F883206928B12E46A4
:102E60005FF0000584F8748010E00026FAE7802106
:102E7000204600F069FEB8B9C6B116F8010B21680A
:102E80000885B4F85200401EA4F85200B4F852006D
:102E90004B464FF0000200970028E8D14FF0400168
:102EA000204600F051FE30B10320D4E735F8020B84
:102EB000C0F30800E3E72020A0670020CBE7022052
:102EC000C9E7000070B50446806F20283CD169B383
:102ED00062B394F87400012836D0012084F874009D
:102EE000E164A4F85020A4F852200025C4F88050D2
:102EF0002120A067E06ED8B114498162E16E1448C8
:102F00001346C862E16E13480863E06E45632668A5
:102F1000E16C06F12802E06EFEF7E9F840B11020FE
:102F2000C4F8800004F8745F20206060012070BD48
:102F300021684020086284F874502068816841F05C
:102F400080018160002070BD022070BDCB3600087A
:102F5000F9360008E335000870477047FEE7F0EEE9
:102F6000401A90ED000AD0ED040A70EE200AC0ED80
:102F7000010A90ED050A30EE800A80EE801A80ED9D
:102F8000031A90ED020A71EEC01A01EE210AF7EE63
:102F9000001A31EEC11A80ED020A61EE200AC0ED7E
:102FA000000A704770B586B018216846FDF7E6F94B
:102FB000254824490024C0E90014012505618460E6
:102FC000457680F82040C0E90A540426C661C460F2
:102FD00080F830500821416104764463FDF7AEFD6E
:102FE00008B1FDF71BFB0720CDE902040095019510
:102FF0000494694614480594FDF7D2FB08B1FDF727
:103000000DFB02200090019069460F48FDF7C8FBB8
:1030100008B1FDF703FB03200090019069460A48C0
:10302000FDF7BEFB08B1FDF7F9FA1220CDE9000665
:1030300069460548FDF7B4FB002801D0FDF7EEFA1C
:1030400006B070BD00010050A8010020114808B56D
:10305000416941F002014161416901F002010091C1
:10306000416941F0010141614069002200F0010025
:10307000009011460E20FEF7BBFA0E20FEF7AAFACA
:10308000002211461120FEF7B3FABDE808401120D6
:10309000FEF7A0BA001002402DE9F04387B01421DA
:1030A0006846FDF76BF93448416941F4800141619C
:1030B000416901F480010591416941F400314161A8
:1030C000416901F400310591416941F48021416178
:1030D000416901F480210591416941F40021416178
:1030E00040694FF0904700F4002005900022032132
:1030F0003846FEF7DDF9DFF8848000224FF45051A6
:103100004046FEF7D5F901224FF440414046FEF714
:10311000CFF9DFF86C904FF48056002231464846D4
:10312000FEF7C6F90320009001250024CDE90154E3
:10313000694638460394FEF7D7F84FF47440009080
:10314000CDE90154694640460394FEF7CDF8E80303
:10315000CDE900040220029069463846FEF7C4F823
:103160000096CDE90154694648460394FEF7BCF841
:1031700007B0BDE8F08300000010024000040048E2
:10318000000800480A4810B508490160062141605E
:1031900040F6FF71C1608160FEF796F9002803D008
:1031A000BDE81040FDF73ABA10BD00000030004005
:1031B0003C02002010B588B0002417480094019408
:1031C000029403940494059412490694016040F615
:1031D0000F61C0E901142321C0E903148461FEF7E3
:1031E000A5FF08B1FDF71AFA4FF480500090694628
:1031F0000948FFF727F808B1FDF710FA049404A96D
:1032000005480694FEF74AFF002801D0FDF706FAAC
:1032100008B010BD000800404C0200200F4810B557
:103220000D4901604FF4E13141604FF480518160FC
:1032300000214FF48062C0E903120C22C0E905218D
:10324000C16101624162FFF75BFC002803D0BDE869
:103250001040FDF7E3B910BD00380140980200208E
:103260000F4810B50D4901604FF4E1314160002174
:1032700081600C22C160C0E904128161C1610162F8
:103280000821416209034163FFF73AFC002803D09B
:10329000BDE81040FDF7C2B910BD00000044004079
:1032A0001C0300200D4810B50B4901604FF4E131BB
:1032B0004160002181600C22C160C0E9041281617B
:1032C000C16101624162FFF71BFC002803D0BDE829
:1032D0001040FDF7A3B910BD00480040A003002036
:1032E000FEE7FEE770477047FEF724B930B59FB0A0
:1032F00028210FA8FDF742F8142119A8FDF73EF880
:103300003C216846FDF73AF8092001210F904FF45F
:10331000803000241591CDE910040225CDE9165026
:1033200013914FF4E01018900FA8FEF7BBFB08B103
:1033300072B6FEE70F20CDE919054FF48060CDE9A4
:103340001B40022119A81D94FEF7A2FA08B172B61B
:10335000FEE78720009004944FF480700990029457
:1033600003946846FEF788F9002801D072B6FEE79C
:103370001FB030BD0248016841F470010160704720
:1033800088ED00E00148FEF7CCBF00004C020020B1
:103390002DE9F0430268234B234D244E244C4FF07B
:1033A0008049984207D0484505D0A84203D0B04292
:1033B00001D0A04203D122F070074A683A431D4F62
:1033C000DFF874C0DFF8748098420DD048450BD008
:1033D000A84209D0B04207D0A04205D0B84203D0DD
:1033E000604501D0404503D122F44075CA682A43A4
:1033F0004D6922F080022A4302608A68C2620A682C
:103400008262984207D0A04205D0B84203D06045FE
:1034100001D0404501D10969016301214161BDE845
:10342000F0830000002C0140000400400008004030
:103430000034014000400140004401400048014088
:1034400010B5846842EA032224F47F440A432243ED
:10345000826010BD826822F070020A4342F00701C8
:103460008160704710B5036A046A24F001040462A5
:10347000846924F0F00444EA021423F00A020A43A7
:103480008461026210BD10B5036A23F01003036269
:103490008369046A23F4704343EA023224F0A003F0
:1034A00043EA01118261016210BD90F82410C9073E
:1034B00006D001684A68836A22F400321A434A60DF
:1034C00090F82410890706D501684A68C36A22F477
:1034D00080321A434A6090F82410490706D50168E3
:1034E0004A68036B22F480221A434A6090F8241041
:1034F000090706D501684A68436B22F400421A4363
:103500004A6090F82410C90606D501688A68836B62
:1035100022F480521A438A6090F82410890606D556
:1035200001688A68C36B22F400521A438A6090F8DB
:103530002410490611D501684A68036C22F48012F0
:103540001A434A60016CB1F5801F06D101684A68D0
:10355000436C22F4C0021A434A6090F82410090612
:1035600006D501684A68806C22F4002202434A6052
:103570007047F8B500260446C0F88060FDF79EFF4E
:103580000546206800686FF07E47000708D52B4687
:1035900000224FF400112046009700F0D5FA60B9E0
:1035A0002068006840070AD52B4600224FF48001AE
:1035B0002046009700F0C8FA08B10320F8BD20208B
:1035C000A067E067266684F874600020F8BD10B537
:1035D000406A0021A0F85A10A0F85210FFF766F9CF
:1035E00010BD70B5446AA06FE56F216889684FF01F
:1035F0000006090606D5212804D1A4F85260204609
:1036000000F097F820688068400606D5222D04D186
:10361000A4F85A60204600F074F8D4F8800040F016
:103620001000C4F880002046FFF740F970BD10B5C7
:103630000146406A896920291BD00021A0F85A1050
:1036400001680A6822F480720A6001688A6822F0C0
:1036500001028A6001688A6822F040028A602021A3
:10366000C167016E012904D101680A6822F01002C5
:103670000A60016E012902D0FFF796FB10BDB0F879
:103680005810FFF763F810BD10B5406A016E0129AC
:1036900002D0FFF7B9FB10BDB0F858104908FFF78A
:1036A00055F810BD10B5406A0021A0F85A10036803
:1036B0000F221A620268936943F008039361202283
:1036C000C2670166FFF7ABF810BD10B50146406A4E
:1036D000896920290DD00021A0F8521001688A685C
:1036E00022F080028A600068016841F040010160B8
:1036F00010BDFFF731FC10BD10B5406AFFF72DFC7F
:1037000010BD01680A6822F490720A6001688A6834
:1037100022F001028A60016E012904D101680A6861
:1037200022F010020A602021C16700210166416673
:10373000704701680A6822F0C0020A602021816790
:10374000704770B5B0F85C10C26F04460068222A5A
:1037500004D0816941F00801816170BD808C626D87
:1037600008401080606D801C6065B4F85A00401EEF
:10377000A4F85A00B4F85A000028EED12068016875
:1037800021F4907101602068816821F0010181605D
:103790002020E06700256566206E012804D02046C1
:1037A000FFF702FB256670BD2068016821F010015B
:1037B0000160B4F858102046FEF7C8FFF2E7000099
:1037C0000148FFF781B80000980200200148FFF788
:1037D0007BB800001C0300200148FFF775B800000B
:1037E000A0030020FEE720F00100008870474FF0A2
:1037F0004070E1EE100A704700000000010203046F
:10380000FE3218CB70B5B0F85C10C26F0446006889
:10381000222A04D0816941F00801816170BD808C49
:103820000840616D0870606D401C6065B4F85A0016
:10383000401EA4F85A00B4F85A000028EED12068BF
:10384000016821F4907101602068816821F0010114
:1038500081602020E06700256566206E012804D085
:103860002046FFF7A1FA256670BD2068016821F0A7
:1038700010010160B4F858102046FEF767FFF2E728
:1038800070B5044680682169E269084361690025D2
:10389000114322680843116849F20C6399430143BC
:1038A000116020684168E26821F440511143416091
:1038B000216AA06901432068826822F430620A43C9
:1038C00082605A4A20685A4990420CD1086B10F025
:1038D000030006D001285FD002285FD0032845D11D
:1038E00058E0012143E0534A90420DD1086B10F497
:1038F00040304DD0B0F5803F4ED0B0F5003F4DD0B8
:10390000B0F5403F32D145E04B4A90420DD1086BB3
:1039100010F440203CD0B0F5802F3DD0B0F5002F02
:103920003CD0B0F5402F21D134E0444A90420DD133
:10393000086B10F440102BD0B0F5801F2CD0B0F5E0
:10394000001F2BD0B0F5401F10D123E03C4A90421D
:103950000CD1086B10F440001AD0B0F5800F1BD0CA
:10396000B0F5000F1AD0B0F5400F13D01021E36965
:103970004FF40040334A4FF6EF7683422ED10929A7
:103980004AD2DFE801F00D101349154949491800E2
:103990000021ECE70221EAE70421E8E70821E6E755
:1039A000FEF71AF806E0FEF72FF803E0104602E0F3
:1039B000FEF742F888B34100606801EB5001B1FBAB
:1039C000F0F081B2A1F11000B04225D84FF6F072AC
:1039D00001EA0200C1F3420108431FE009291BD29A
:1039E000DFE801F005080B1A0D1A1A1A1000FDF78E
:1039F000F3FF06E0FEF708F803E0104602E0FEF7EA
:103A00001BF850B1616800EB5100B0FBF1F080B2DF
:103A1000A0F11001B14201D9012501E02168C8607F
:103A200000206066A066284670BD00000038014096
:103A3000001002400044004000480040004C00409C
:103A40000050004000127A0070B54165A0F858207F
:103A500000250446C0F880502220E067206FD8B1CE
:103A600017498162216F17481346C862216F1648B3
:103A70000863206F4563666D216832462431206FEC
:103A8000FDF735FB40B11020C4F8800004F8745FE6
:103A900020206060012070BD84F8745020680168A7
:103AA00041F4807101602068816841F0010181600A
:103AB0002068816841F040018160002070BD0000F5
:103AC0002F36000889360008E335000810B5416537
:103AD000A0F85820A0F85A200021416682684FF4CF
:103AE0008054FF23A24204D1026922BB40F2FF129C
:103AF0001EE0D2B1A0F85C10C0F880102222C2678C
:103B00000268936843F0010393608268A24201D186
:103B100002699AB10A4A426680F874100068016826
:103B200041F490710160002010BD02691AB17F223A
:103B3000A0F85C20E0E7A0F85C30DDE7014AEAE7A6
:103B400005380008433700082DE9F0479A46174624
:103B50000E4604464FF000094FF02008089D39E05A
:103B6000681C37D0FDF7AAFCA0EB0A00A84222D8B7
:103B70000DB32068016849072CD5C069C043000512
:103B800028D421684FF4006008622068016821F49D
:103B9000D07101602068816821F001018160C4F862
:103BA0007880C4F87C80C4F8808000BF84F874906A
:103BB0000320BDE8F0872068016821F4D07101601E
:103BC0002068816821F001018160C4F87880C4F820
:103BD0007C80EBE72068C06936EA000004D0002052
:103BE000B842BDD00020E4E70120F9E70907090E3B
:103BF000002804DB00F1E02080F80014704700F09A
:103C00000F0000F1E02080F8141D704743F6982162
:103C10004143A0F6E770404291FBF0F10848814231
:103C200001D9FF207047074A002000BF52F820301A
:103C30008B42F7D3401CC0B2FF28F7D37047000077
:103C40007BF131007841000870B53F24204A214DB6
:103C50009FED212ADFED212A0021D0882B8896882C
:103C600000EE106AF8EE400A00EE103AB8EE400A94
:103C700020EE800A60EE020A00EE100AB8EE401A4A
:103C800080EE810A20EE220ABCEEC00A10EE100A75
:103C900080B200EE100A0E48B8EE400A2030FFF75E
:103CA0005EF9BCEEC00A491C89B210EE100A642904
:103CB00083B2D2D300200A4903E0401C80B2A04264
:103CC00003D231F810209A42F7D8401C80B270BD60
:103CD00014000020BAF7FF1F00404E450000803955
:103CE0003C4500087FB50D4620F00104FDF7E8FAD9
:103CF00000208DE83100039003A96846FDF742FAE1
:103D0000FDF794FA7FBD70B50D4620F00104FDF774
:103D1000D7FA24F001000088A0F57F41FF3905D1D2
:103D20002A46002321460120FDF78AFABDE87040AB
:103D3000FDF77CBA2DED028B84B0FDF703FCFFF795
:103D4000D5FAFFF7A9F9FFF781F9FFF72BF9FFF78C
:103D500065FAFFF785FAFFF7A5FAFFF72BFAFFF7E9
:103D600011FA4FF47A70FDF7FBF94FF40040FFF7BA
:103D70003AFDF34C00212070F248FCF7C5FC042208
:103D800004F11401EF48FDF747F84FF48056002284
:103D90003146ED48FDF78CFB0A22EC49EC48FEF772
:103DA000B0FCEC48FEF73CFD0122E11CE948FEF7BF
:103DB000DCFFE948FEF70AFAFFF746FF00F03F0094
:103DC0006070E16800F01F00087094F9010082063D
:103DD00000F01F0000D54042607094F800200020E1
:103DE00000EB800301EB8303401CC0B21A7702286A
:103DF000F6D3DFF858B3DFF848830BF10A0B08F16C
:103E00000808B1469FEDD58ADFEDD58A4FF0C80A84
:103E100008F10C07A088401CA0802820FDF7A0F91D
:103E200000258DF80450ADF80850ADF80050CD488D
:103E3000FDF779FB94F9000094F90110401C8842C9
:103E40004FF0010206D1C84E91033046FDF730FB1A
:103E5000710107E0C44E4FF400413046FDF728FBE6
:103E60004FF480413046FDF71BFBC048FEF799FC3C
:103E7000B64928220A31BD48FEF758FF9BF80000DA
:103E80005E4655280BD17078AA2808D1B078BB2897
:103E900005D1A022B548E168FFF714F8B570207984
:103EA000E26800F0010000EB800102EB810191F873
:103EB0002010090611D518F8000000060DD40121C4
:103EC000CE033046FFF70EFF94F90100401E81B289
:103ED0003046FFF718FFFDF7BDFB2079E26800F0E0
:103EE000010101EB810002EB800090F8203008F81E
:103EF000013090F821100906417E02D541F0800181
:103F000001E021F0800141769748143001684CF6B9
:103F1000FF721140ADF80010217901F0010209EBA8
:103F20000231BDF80020114301600120FDF718F9AE
:103F30008F49F88809883A8800EE102AF8EE400A7E
:103F400000EE101AB8EE400A20EE800A60EE080A71
:103F500000EE100AB8EE401A80EE810A20EE280A20
:103F6000BCEEC00A10EE100AADF80000BDF800105B
:103F700040F6C4108142BDF80000A0F6C41002D97A
:103F8000C0EB001101E0A0EB001191FBFAF0ADF8DD
:103F9000000020796A4900F00100243140F2F31357
:103FA00051F820205A435E1CB2FBF6F2BDF80030F7
:103FB0001A4441F82020B2FBF6F1ADF80010BDF82C
:103FC0000010A02902D9FF21ADF80010BDF80010A3
:103FD000C0F10200E26800EB800002EB8000817615
:103FE0007888ADF80000BDF80000FFF70FFE8DF8EF
:103FF00004002079524900F0010010319DF804C0FE
:1040000031F8102002EB421202EB42036422B3FBB0
:10401000F2F363449BB221F81030B3FBF2F18DF858
:1040200004109DF80410FD2902D9FF218DF8041019
:104030009DF80420E16800EB800001EB8000C2766F
:10404000207900F07F00ADF80800BDF80800402896
:1040500001D3012000E000208DF804004FF09040D3
:1040600042694FF6FC731A40ADF80020BDF80020FD
:104070009DF804305B1C1A434261E088ADF80000F3
:10408000E580BDF8080000F03F000528FFF4C2AE4F
:10409000BDF8000028B1BDF800004A2803D94A2025
:1040A00006E02A2004E0BDF800002D2802D22D20D1
:1040B000ADF80000BDF80000DFED2E0A4A3800EE32
:1040C000100AB8EEC00A20EE200AFBEE0D0A80EEC0
:1040D000201ABCEEC10A10EE100AADF80000184814
:1040E0009DF804202C3040F2F31350F822205A435C
:1040F000B2FBF6F2BDF800301A449DF8043040F8E7
:1041000023209DF8042050F82200B0FBF6F0ADF813
:104110000000BDF80000FA2802D9FF20ADF8000029
:10412000BDF800009DF8042002EB820201EB820141
:1041300008228877024906481C31FEF7C3FE69E66B
:1041400000000020A8010020000800485C000020BA
:104150001C030020A00300204C0200200040CE459C
:10416000000080393C020020000400489802002032
:10417000BAF7FF1F00007A437BF1310084BB2E00A9
:1041800007C02B0079FA2800B1662600DE00240063
:1041900082C5210068B11F009BC11D0068F31B0090
:1041A00051441A000CB218007C3A1700B3DB15001A
:1041B000E49314006C611300C442120085361100B0
:1041C000633B10002D500F00C7730E002CA50D008F
:1041D00069E30C009D2D0C00FA820B00C0E20A007E
:1041E0003A4C0A00C6BE0900C8390900B2BC080032
:1041F000024708003AD80700EA6F0700A70D07003A
:104200000EB10600C359060071070600C9B90500C2
:104210007F7005004E2B0500F6E904003BAC04005E
:10422000E3710400BC3A0400930604003BD503008C
:1042300089A60300547A030078500300D1280300B4
:104240003E030300A1DF0200DCBD0200D59D020099
:10425000737F02009C6202003C4702003D2D020079
:104260008B14020015FD0100C8E6010095D1010084
:104270006BBD01003EAA0100FE970100A08601006F
:104280001676010057660100575701000D490100DD
:104290006E3B0100722E0100102201004116010048
:1042A000FD0A01003D000100FAF500002DEC0000C0
:1042B000D2E20000E2D9000058D100002FC900006E
:1042C00062C10000ECB90000CAB20000F7AB000008
:1042D00070A50000319F0000369900007C9300001B
:1042E000008E0000C0880000B8830000E57E00005A
:1042F000467A0000D875000099710000866D0000B4
:104300009D690000DD65000044620000D05E000091
:104310007F5B0000505800004155000051520000E2
:104320007E4F0000C84C00002D4A0000AB47000043
:1043300042450000F1420000B7400000923E0000FC
:10434000813C0000853A00009C380000C536000022
:10435000FF3400004A330000A63100001030000096
:104360008A2E0000112D0000A72B0000492A000012
:10437000F8280000B2270000792600004A25000036
:10438000262400000C230000FD210000F620000080
:10439000F91F0000041F0000181E0000341D00005B
:1043A000571C0000821B0000B41A0000ED19000029
:1043B0002D19000073180000C0170000121700002C
:1043C0006A160000C71500002A15000092140000AC
:1043D000FE13000070130000E612000060120000DF
:1043E000DF11000062110000E910000073100000EE
:1043F00002100000930F0000290F0000C10E000002
:104400005D0E0000FB0D00009D0D0000420D000040
:10441000E90C0000930C0000400C0000EF0B0000C2
:10442000A10B0000540B00000B0B0000C30A00009E
:104430007D0A00003A0A0000F8090000B8090000EF
:104440007B0900003F09000004090000CC080000BF
:10445000950800005F0800002B080000F907000025
:10446000C807000098070000690700003C0700002B
:1044700010070000E6060000BC06000094060000DD
:104480006D0600004706000021060000FD05000043
:10449000DA050000B8050000970500007605000069
:1044A00057050000380500001A050000FD04000053
:1044B000E0040000C5040000AA040000900400000D
:1044C000760400005D040000450400002D04000097
:1044D0001604000000040000EA030000D4030000FA
:1044E000C0030000AB03000097030000840300003A
:1044F000710300005F0300004D0300003B03000058
:104500002A0300001A0300000A030000FA02000058
:10451000EA020000DB020000CC020000BE02000044
:10452000B0020000A2020000950200008802000014
:104530007B0200006E02000062020000C709A509AC
:104540008309610940091E09FC08DA08B8089608C1
:104550007408530831080F08ED07CB07A907870730
:104560006607440722070007DE06BC069A0679069E
:10457000570635061306F105CF05AD058B056A050F
:10458000480526050405E204C0049E047D045B047E
:1045900039041704F503D303B10390036E034C03EE
:1045A0002A030803E602C402A20281025F023D025E
:1045B0001B02F901D701B5019401020304050607A6
:1045C00008090A0B0C0D0E0F10100102030405065A
:1045D0000708090A0B0C0D0E0F1000000000000068
:1045E0000000010203040607080900000C46000849
:1045F000000000205C000000C401000868460008BC
:104600005C0000205C150000E001000800000000D4
:104610000000000000000000060100200000000073
:104620000000000000000000010300000001840AF7
:10463000000000000000000000000000000000007A
:104640000000803F000000000000000000000000AB
:104650006F12833ACDCCCC3D010000001000000069
:084660000000000000127A00C6
:040000050800018965
:00000001FF
